:04000000B60192288B
:100008000800A7008713071307138316871307131E
:100018000713F030870583122708B61831283A30BD
:10002800A100983079203330A60046201330A10073
:100038008830792046206430782046206430782043
:100048002230A6004620283030200C3030200630E0
:100058003020B614270831283614A600361C3F284D
:100068000713033C031C442844200730A100D03068
:100078007920031408003614FE3C03198D2807174D
:10008800A60E361C36108717F030870526080F395C
:1000980087048713A60E36184628323078200314B2
:1000A800080003178D0083168C130C1483120C0898
:1000B8008D2803178C0083168C130C1555308D0072
:1000C800AA308D008C148C1867280C118D28A30178
:1000D800A200FF30A207031CA307031C8D280330CE
:1000E800A100DF3079206D28A101E83EA000A10918
:1000F800FC30031C8228A00703187F28A00764008F
:10010800A10F7F2820188828A01C8C2800008C2884
:100118000800831303138312640008008B178A11E5
:100128000A129B288B1B08008A110A1232298A019D
:1001380096208316890183128A01962083167030CF
:10014800860083128A019620831607309F00831247
:100158008A0196200F3086008A019620831681171F
:1001680083128A01962088308B008A019620C60166
:100178008A0196200130A300F4308A016C208A019C
:100188009620FE308A01052001308A0105202030A2
:100198008A01052020308A01052020308A010520A7
:1001A80020308A0105202D308A0105202D308A0152
:1001B800052020308A01052078308A010520783012
:1001C8008A01052020308A0105202D308A0105206A
:1001D8002D308A0105208A019620FE308A010520EB
:1001E800C0308A01052020308A01052020308A018C
:1001F800052020308A01052020308A0105202D3075
:100208008A0105202D308A01052020308A01052029
:1002180078308A01052078308A01052020308A014B
:1002280005202D308A0105202D308A0105208A01FC
:1002380096200130A300F4308A016C2000000000F1
:100248000000000000000000000000008A01962065
:1002580088308B008A0196208A0122290F308A0172
:100268006B20C4010B10FE308A01052001308A0181
:10027800052053308A01052069308A01052066303F
:100288008A01052072308A01052065308A0105201F
:100298006E308A01052069308A0105207A308A018A
:1002A800052069308A010520FE308A010520C0300A
:1002B8008A01052047308A01052069308A01052016
:1002C80072308A01052069308A0105206E308A0162
:1002D800052069308A0105207A308A0105200F300F
:1002E80086008A110A12C82214308A016B200F3046
:1002F8000606C90064008A110A1203197829143005
:100308008A016B2070300606C90064008A110A123F
:10031800031978290130860064008A110A12061A26
:10032800A22964008A110A12861AA22964008A1175
:100338000A12061BA2298A110A12A5298A110A1271
:10034800E9290230860064008A110A12061AB929BE
:1003580064008A110A12861AB92964008A110A12DD
:10036800061BB9298A110A12BC298A110A12E9291D
:100378000430860064008A110A12061AD029640023
:100388008A110A12861AD02964008A110A12061BD9
:10039800D0298A110A12D3298A110A12E9290830A8
:1003A800860064008A110A12061AE62964008A1176
:1003B8000A12861AE62964008A110A12061BE6291F
:1003C8008A018E298A110A12E9290608C800C30180
:1003D8008A110A1276246400490848028A110A120E
:1003E8000319032AC30A64000A3043028A110A1255
:1003F800031C012AC3018A018E298A01EC296400A1
:100408000A3043028A110A120318732944083C3E31
:10041800840043088000C40A64004408013C8A112F
:100428000A12031D232AFE308A01052001308A01A1
:1004380005202A308A0105208A110A12262A2A3024
:100448008A01052064004408053C8A110A12031D2C
:100458003D2AC301C40164008A110A12C61B3A2A44
:100468008A110A12402A8A110A123D2A8A110A128E
:10047800EB2BC3018A017329C50100304507B2007F
:10048800B301B30D32088A015520C90045083C3E26
:1004980084000008B2006400320849028A110A1276
:1004A800031D662AC50A64004508053C8A110A121C
:1004B800031D642A8A110A12DD2A8A110A12662A81
:1004C8008A01412A8A110A12692AFE308A01052006
:1004D80001308A01052059308A01052041308A01FE
:1004E80005204E308A0105204C308A01052049300C
:1004F8008A01052053308A01052020308A01052011
:1005080053308A01052069308A01052066308A0146
:10051800052072308A01052065308A010520FE30E9
:100528008A010520C0308A01052054308A0105203F
:1005380045308A0105204B308A01052052308A0156
:10054800052041308A01052052308A0105202030DB
:100558008A01052044308A01052065308A0105207A
:100568006E308A01052079308A01052069308A01B8
:1005780005206E308A0105200B30A300B8308A01AF
:100588006C208A110A12652C0A308A016B206400DB
:100598008A110A12061ADB2A64008A110A12861ABC
:1005A800DB2A64008A110A12061BDB2A08008A016A
:1005B800C82AFE308A01052001308A0105205430FE
:1005C8008A01052065308A01052072308A010520DC
:1005D80063308A01052069308A01052068308A0164
:1005E800052069308A0105206E308A0105206930AE
:1005F8008A0105207A308A01052028308A010520E1
:1006080030308A0105202C308A01052031308A01DA
:10061800052029308A0105200F3086000730A30005
:10062800D0308A016C2064008A110A12061A2C2B19
:1006380064008A110A12861A262B8A01172B8A113E
:100648000A12292B8A110A12922B8A110A122F2BAD
:100658008A110A122F2BFE308A01052001308A01E7
:10066800052047308A01052069308A01052072304B
:100678008A01052069308A01052073308A01052026
:1006880020308A01052047308A01052065308A011B
:10069800052063308A01052065308A010520723003
:1006A8008A0105206C308A01052069308A010520FD
:1006B8000330A300E8308A016C200914FE308A0157
:1006C800052001308A01052069308A01052079302A
:1006D8008A01052069308A01052020308A01052019
:1006E80020308A01052047308A01052075308A01AB
:1006F80005206E308A0105206C308A01052065309E
:100708008A01052072308A0105200F30A300A0302D
:100718008A016C2009108A110A12652CFE308A01A0
:10072800052001308A01052059308A0105206530ED
:100738008A0105206E308A01052069308A0105206A
:1007480020308A01052053308A01052069308A014A
:10075800052066308A01052072308A01052065303F
:100768008A0105206E308A01052069308A0105203A
:100778007A308A01052069308A010520FE308A0115
:100788000520C0308A01052020308A01052020304C
:100798008A01052047308A01052069308A01052031
:1007A80072308A01052069308A0105206E308A017D
:1007B800052069308A0105207A308A010520C6178C
:1007C8000130A300F4308A016C208A017329C50125
:1007D8006400053045028A110A120318092C0030FA
:1007E8004507B200B301B30D45083C3E840000083C
:1007F800B400320803178D00031334088A015D2002
:10080800C50A8A110A12031DEC2BFE308A01052045
:1008180001308A01052059308A01052065308A0196
:1008280005206E308A01052069308A0105202030B4
:100838008A01052053308A01052069308A01052084
:1008480066308A01052072308A01052065308A01E8
:1008580005206E308A01052069308A0105207A302A
:100868008A010520FE308A010520C0308A01052052
:100878004B308A01052041308A01052059308A0110
:10088800052049308A01052054308A01052020308E
:100898008A01052045308A01052064308A01052037
:1008A80069308A0105206C308A01052064308A018C
:1008B800052069308A0105200B30A300B8308A0171
:1008C8006C20FE308A01052001308A010520C6010E
:1008D8000F3086008B0164308A016B200B108B1758
:1008E8008A01BC2843080B3C8A110A12031C932C6A
:1008F8008A110A128324C9008A110A12932C04301F
:100908008A004308820711342134413412342234D6
:100918004234143424344434183428344834080015
:0A0928008A01962063008A01962CD4
:02400E00713D02
:0A42000001000700000006000100A5
:00000001FF
